:100000000C94CB050C94E8050C94E8050C94E805D9
:100010000C94E8050C94E8050C94E8050C94E805AC
:100020000C94E8050C94E8050C94E3270C94B5288F
:100030000C94F6210C94E8050C94E8050C94E80562
:100040000C94E8050C94E8050C94E8050C94E8057C
:100050000C94E8050C947E220C94E8050C94E805B9
:100060000C94E8050C94E8050C94E8050C94E8055C
:100070000C94E8050C94E8050C94E8050C94E8054C
:100080000C94E8050C94E8050C94E8050C94E8053C
:100090000C94E8050C94E8050C94E8050C94E8052C
:1000A0000C94E8050C94E8050C94E805B909B90925
:1000B000E509E5094D0A6B0A830B830B760A0F0BE2
:1000C000200B200B241E121E2B1E9D1DD81ED81E79
:1000D0000F1ED81ED81E581ED81E6C1EB81ED81E45
:1000E000D81ED81ED81E8C1ED81ED81E891ED81EFB
:1000F000441ED81ED81ED21ED21ED21ED21ED21E02
:10010000D21ED21ED21ED21ED41ED81E241E071EE0
:10011000D81ED81ED81ED81ED81ED81ED81ED81E2F
:10012000D81ED81ED41ED81ED81E0F1ED81ED01EF4
:10013000D01ED01ED01ED01ED01ED01ED01ED01E4F
:10014000D41E22294929412A4929412A9529B82919
:10015000412A0F2A1E2A3F003E003D003C003B0082
:100160003A00E3002C00E0004600E50038003700CC
:100170003600100011000500190006001B001D00CC
:10018000E200E1003500340033000F000E000D00E6
:100190000B000A00090007001600040031002800C7
:1001A00030002F00130012000C0018001C00170074
:1001B000150008001A0014002B002A002E002D0044
:1001C0002700260025002400230022002100200013
:1001D0001F001E00290000000000000000000000B9
:1001E0004C0049004E0051004D0000004F004800F7
:1001F000500000004B0052004A00470053004300EB
:1002000042004100400044454255473A206469732A
:1002100061626C65642E0A0044454255473A206588
:100220006E61626C65642E0A000A00253032580047
:100230006C65645F7461736B3A20004F6E65736820
:100240006F743A206163746976653A2025640A0008
:100250000A0025303862003A200025303258000A62
:10026000722F632030313233343536370A00290A91
:10027000002575002F002575005D280025640020ED
:1002800000256400200025640020002564007C0017
:1002900025303258006D6F7573656B6579205B6230
:1002A000746E7C782079207620685D287265702FC6
:1002B00061636C293A205B00313A0964656C6179AD
:1002C000282A31306D73293A2025750A323A096996
:1002D0006E74657276616C286D73293A2025750AF3
:1002E000333A096D61785F73706565643A202575EE
:1002F0000A343A0974696D655F746F5F6D61783AAD
:100300002025750A353A09776865656C5F6D6178F7
:100310005F73706565643A2025750A363A09776817
:1003200065656C5F74696D655F746F5F6D61783A68
:100330002025750A00703A097072696E7420766122
:100340006C7565730A643A09736574206465666147
:10035000756C74730A75703A092B310A646E3A0928
:100360002D310A6C743A092B31300A72743A092D16
:1003700031300A4553432F713A09717569740A0A7D
:100380007370656564203D2064656C7461202A206B
:100390006D61785F7370656564202A2028726570CE
:1003A000656174202F2074696D655F746F5F6D6186
:1003B00078290A77686572652064656C74613A20F3
:1003C000637572736F723D25642C20776865656C68
:1003D0003D25640A53656520687474703A2F2F6553
:1003E0006E2E77696B6970656469612E6F72672F15
:1003F00077696B692F4D6F7573655F6B6579730AEC
:10040000004D3E20004D25753A25733E20003F0AE1
:10041000003D2025750A003F0A0064656661756C21
:1004200074730A0025750A003F0A000A092D205638
:10043000616C756573202D0A00710A000A092D2070
:100440004D6F7573656B6579202D0A003F00433E43
:1004500020004C25640A000A092D2053746174752C
:1004600073202D0A686F73745F6B6579626F6172B8
:10047000645F6C65647328293A20253032580A6B12
:100480006579626F6172645F70726F746F636F6CB5
:100490003A20253032580A6B6579626F6172645F69
:1004A00069646C653A20253032580A6B65796D6154
:1004B000705F636F6E6669672E6E6B726F3A202590
:1004C0003032580A74696D65725F726561643332E7
:1004D00028293A202530386C580A000A092D205660
:1004E000657273696F6E202D0A5649443A20307840
:1004F00046454544284E6F626F647929205049442F
:100500003A2030783630363028726574726F5F72F8
:100510006566697429205645523A2030783030306B
:10052000310A4255494C443A20202846656220321F
:10053000372032303232290A4F5054494F4E533A05
:10054000204C554641204D4F5553454B455920456C
:10055000585452414B455920434F4E534F4C452020
:10056000434F4D4D414E44204E4B524F203531327A
:100570000A4743433A20352E342E30204156522D1F
:100580004C4942433A20322E302E30204156525FA1
:10059000415243483A20617672350A000A092D20FB
:1005A000436F6E736F6C65202D0A4553432F713A6C
:1005B00009717569740A6D3A096D6F7573656B65BC
:1005C000790A000A092D204D61676963202D0A44CC
:1005D0003A094465627567204D65737361676520EC
:1005E000546F67676C650A583A094D61747269788F
:1005F000204465627567204D6F646520546F67679E
:100600006C65202D2053686F77206B65797072655B
:100610007373657320696E206D61747269782067E9
:100620007269640A4B3A094B6579626F61726420A2
:10063000446562756720546F67676C65202D205391
:10064000686F77206B65797072657373207265705F
:100650006F72740A4D3A094465627567204D6F7573
:10066000736520546F67676C650A563A0956657260
:1006700073696F6E0A533A095374617475730A4350
:100680003A09416374697661746520436F6E736FD4
:100690006C65204D6F64650A46312D4631303A094C
:1006A00053776974636820746F204C617965722098
:1006B000302D392028463130203D204C30290A3059
:1006C0002D393A0953776974636820746F204C613F
:1006D00079657220302D390A47524156453A0953FF
:1006E000776974636820746F204C6179657220307B
:1006F0002028616C7465726E617465290A423A093A
:100700004A756D7020746F20426F6F746C6F6164F6
:1007100065720A4553433A094A756D7020746F201B
:10072000426F6F746C6F616465722028616C7465D0
:10073000726E617465290A453A095072696E7420B7
:10074000454550524F4D2053657474696E67730A66
:100750004253504143453A09436C65617220454517
:1007600050524F4D0A4E3A094E4B524F20546F672C
:10077000676C650A006B65796D61705F636F6E66AB
:1007800069672E7261773A20253032580A2E7377C6
:1007900061705F636F6E74726F6C5F636170736CB6
:1007A0006F636B3A2025750A2E636170736C6F63FB
:1007B0006B5F746F5F636F6E74726F6C3A20257538
:1007C0000A2E737761705F6C63746C5F6C67756918
:1007D0003A2025750A2E737761705F7263746C5FBF
:1007E000726775693A2025750A2E737761705F6CA0
:1007F000616C745F6C6775693A2025750A2E737792
:1008000061705F72616C745F726775693A202575FB
:100810000A2E6E6F5F6775693A2025750A2E737709
:1008200061705F67726176655F6573633A202575F5
:100830000A2E737761705F6261636B736C617368BA
:100840005F6261636B73706163653A2025750A2E80
:100850006E6B726F3A2025750A0064656275675F7A
:10086000636F6E6669672E7261773A202530325861
:100870000A2E656E61626C653A2025750A2E6D61DF
:10088000747269783A2025750A2E6B6579626F61FA
:1008900072643A2025750A2E6D6F7573653A2025AE
:1008A000750A006565636F6E6669673A0A64656616
:1008B00061756C745F6C617965723A2025750A0008
:1008C0003F004E4B524F3A206F66660A004E4B5225
:1008D0004F3A206F6E0A000A6D6F7573653A206F8C
:1008E00066660A000A6D6F7573653A206F6E0A00BE
:1008F0000A6B6579626F6172643A206F66660A00FE
:100900000A6B6579626F6172643A206F6E0A000A41
:100910006D61747269783A206F66660A000A6D61CB
:10092000747269783A206F6E0A000A6465627567AE
:100930003A206F66660A000A64656275673A206F3E
:100940006E0A000A0A4A756D70696E6720746F201E
:10095000626F6F746C6F616465722E2E2E2000437F
:100960003E2000436C656172696E672045455052B8
:100970004F4D0A000A002530325820006B6579621D
:100980006F6172645F7265706F72743A20006465A3
:100990006C5F6B65795F6269743A2063616E27747E
:1009A0002064656C3A20253032580A006164645F27
:1009B0006B65795F6269743A2063616E27742061A8
:1009C00064643A20253032580A005B735D005B573F
:1009D0005D005B535D005B525D005B445D005B430B
:1009E0005D00180372006500740072006F005F0004
:1009F0007200650066006900740000000E034E007E
:100A00006F0062006F0064007900000004030904B5
:100A100009025B00030100A0FA09040000010301C0
:100A2000010009211101000122400007058103088E
:100A30000001090401000103000000092111010067
:100A40000122B6000705820320000109040200020A
:100A50000300000009211101000122220007058383
:100A6000032000010705030320000112010002001A
:100A7000000008EDFE60600100010200010631FF88
:100A80000974A1010975150026FF009520750881DC
:100A9000020976150026FF00952075089102C00511
:100AA000010902A10185020901A100050919012915
:100AB0000815002501950875018102050109300915
:100AC000311581257F950275088106093815812524
:100AD0007F950175088106050C0A38021581257F6E
:100AE000950175088106C0C005010980A101850333
:100AF00019012AB700150126B7009501751081006C
:100B0000C0050C0901A101850419012AA0021501E3
:100B100026A002950175108100C005010906A101FA
:100B20008506050719E029E71500250195087501D7
:100B300081020507190029EF1500250195F07501BF
:100B40008102050819012905950575019102950194
:100B500075039101C005010906A101050719E029E6
:100B6000E715002501950875018102950175088139
:100B7000010507190029FF150026FF0095067508D5
:100B80008100050819012905950575019102950156
:100B900075039101C00011241FBECFEFDAE0DEBF64
:100BA000CDBF11E0A0E0B1E0EEEFF5E502C00590A9
:100BB0000D92AA3FB107D9F723E0AAEFB1E001C037
:100BC0001D92A034B207E1F70E94C6170C94FD2ACB
:100BD0000C940000FF93EF93E091FA01F091FB0178
:100BE000309709F00995EF91FF910895FC018591E7
:100BF000803011F0EFDFFBCF0895FF27E0E230E215
:100C000047FF0CC0419597FF09C0EDE260957095D4
:100C100080959095611D711D811D911D27FF02C05A
:100C2000219530E350E2AA27660F771F881F991F8E
:100C3000AA1FA41710F0A41B63955A95A9F7AA3010
:100C400008F0A95FA05DAF93F3956115710581056B
:100C5000910541F7ED3211F4EF93F395F21718F483
:100C60003F93F395FBCF8F91B5DFFA95E1F70895A8
:100C7000E991F9918591803021F0853219F0AADF50
:100C8000F9CF089520E0E89455915532C1F35033DF
:100C900011F4689455915A3348F4505390F3220F4D
:100CA000022E220F220F200D250FF4CF0EF42195D6
:100CB00089919991533619F3533729F1533559F1E5
:100CC000BC0188279927E8945C3621F48991999191
:100CD00068945591543639F446EF7EF077FF0DC095
:100CE0008FEF9FEF0AC055374AE039F0583540E1A1
:100CF00021F0523642E009F00895FF93EF937DDF33
:100D0000EF91FF91B7CFFF93EF93FC01819180307A
:100D1000B9F360DFFBCFFF93EF9368DFF1CFDF9391
:100D2000CF93CDB7DEB72596A3DFCF91DF9108959E
:100D3000569A5E9A0C94861681FF02C0509A01C0A2
:100D40005098589880FF02C0519A01C05198599804
:100D500082FF02C03E9A01C03E9846980C94A107BB
:100D600081E0089581E008950C94B20608950C94F2
:100D7000B6061F93CF93DF9300D000D01F92CDB75C
:100D8000DEB749835A836B833091FD0189819A8153
:100D9000311114C0662359F0222349F00E94C00D7E
:100DA000182F682F89819A810E94690D03C00E94C3
:100DB000940D182F69817A81812F04C00E94C00D83
:100DC00069817A810F900F900F900F900F90DF91B3
:100DD000CF911F910C940015FC01262F4081518169
:100DE0006281738184810C94B90681E00895CF9368
:100DF000DF93EC0160E00E94EC06BE01DF91CF9131
:100E00000C94B7060C9498060C94841608950E94CE
:100E1000130C0E9406072FEF84E39CE021508040D2
:100E20009040E1F700C000000C94A4220F931F93A0
:100E3000CF93DF938C0161E00E94EC06EC01B801D6
:100E40000E94B406882309F45BC0B801CE010E9459
:100E5000E51F882309F454C0B801CE010E94DE1AB0
:100E6000882309F44DC0B801CE010E94411F882398
:100E700009F446C0F80182818823D9F1CF3D8CE581
:100E8000D80779F140F4C115FCE5DF0791F0C130D6
:100E9000DC4591F02EC0CC35EDE5DE0741F1CD35D6
:100EA000FDE5DF0709F1CB35DD4519F50E94571245
:100EB00020C00E94070724C08091CC02C82FC09593
:100EC000C170C0FB80F98093CC02CC2329F088E16B
:100ED00092E00E94F60514C086E092E00E94F605BA
:100EE00010C00E940B130CC00E944E1202C00E9440
:100EF0005A12C801DF91CF911F910F910C94B00647
:100F0000C0E08C2FDF91CF911F910F9108950E9427
:100F1000D9210C94B0070E94B3070C94DF2182956D
:100F2000982F937344E0949F900111248C7C8695B4
:100F30008695282B822F8575880F2A7A2695822BF5
:100F40000895089581E008950C94A2070895CF9321
:100F5000C82F0E949C068C2F0E94A407CF91089551
:100F600080E00C94A7070E9441200C94A707CF9320
:100F70000E944120C82F8091FC01C81741F1C09305
:100F8000FC018091CC0282FF1EC080FF04C080E380
:100F900092E00E94F6058091CC0280FF0CC01F9267
:100FA000CF938BE292E09F938F930E948F060F90D6
:100FB0000F900F900F908091CC0280FF04C089E2C7
:100FC00092E00E94F6058C2FCF910C94A707CF9149
:100FD0000895CF93DF93CDB7DEB72B970FB6F89474
:100FE000DEBF0FBECDBF4F83588769877A878B8757
:100FF00061110E9486119E012F5F3F4F86E0F9012B
:1010000011928A95E9F785E0FE013796D9010190A2
:101010000D928A95E1F789819A814C815D81452BFA
:1010200031F09F3F31F491E08F3F19F403C091E01C
:1010300001C090E090FF09C049815A816B817C8199
:101040008D819E810E94A71005C0C9010E94F506EE
:101050008111F2CF2B960FB6F894DEBF0FBECDBF35
:10106000DF91CF910895FC01808191810E94020E51
:101070000895CF93882309F4A9C0C82F8238C1F4FA
:101080000E94412081FDA2C069E3809102019091FC
:1010900003010E9494210E94A8112FEF81EE94E099
:1010A000215080409040E1F700C0000069E319C082
:1010B000833801F50E94412080FD88C063E580915E
:1010C0000201909103010E9494210E94A8112FEF28
:1010D00081EE94E0215080409040E1F700C0000094
:1010E00063E580910201909103010E949F21CF91BD
:1010F0000C94A8118438C1F40E94412082FD66C07E
:1011000067E480910201909103010E9494210E9462
:10111000A8112FEF81EE94E0215080409040E1F73C
:1011200000C0000067E4DDCF8CEF8C0F813AF8F44B
:101130008C2F0E94EA1E811149C06C2F8091020100
:10114000909103010E94F220882349F06C2F809136
:101150000201909103010E949F210E94A8116C2F0F
:1011600080910201909103010E949421C0CF80E2FE
:101170008C0F883048F4C77081E001C0880FCA9591
:10118000EAF70E946911B3CFEBE5EC0FE33040F4CE
:10119000F0E0E95BFE4F808190E0CF910C94B020AD
:1011A000E8E5EC0FE73150F4F0E0EE0FFF1FE75EEB
:1011B000FE4F80819181CF910C94C620CD3E30F0BE
:1011C0008C2F0E944B18CF910C941D19CF9108952C
:1011D000882309F464C0823879F40E94412081FF99
:1011E0005EC069E380910201909103010E94942105
:1011F0000E94A81169E310C08338B1F40E94412015
:1012000080FF4DC063E580910201909103010E942F
:1012100094210E94A81163E580910201909103013D
:101220000E949F210C94A811843879F40E944120D7
:1012300082FF35C067E480910201909103010E9412
:1012400094210E94A81167E4E7CF9CEF980F913A90
:1012500010F4682FE1CF90E2980F983050F4877027
:1012600091E001C0990F8A95EAF7892F0E946F11CA
:10127000D9CF9BE5980F933020F480E090E00C9458
:10128000B02098E5980F973120F480E090E00C941E
:10129000C6208D3E20F00E94A6180C941D190895BA
:1012A0001F93CF93DF93182FEB010E9439082097EB
:1012B00041F08FE99FE00197F1F700C0000021970E
:1012C000F6CF812FDF91CF911F910C94E8088933DD
:1012D00019F060E070E002C060E570E00C94500925
:1012E000882321F00E9469110C94A8110895882385
:1012F00021F00E946F110C94A8110895CF92DF92F3
:10130000EF92FF920F931F93CF93DF937C01D62F21
:10131000C72FFC011281058102950F700E945F1199
:101320008823B9F01123A9F08C2F807F803421F01D
:1013300080E28D0F883068F08091180382FD09C02B
:1013400082E00E9408120E945F1191E0D82ED926F7
:1013500001C0D12CCC2EC2948FE0C8228C2D90E0FD
:101360008C30910508F0CFC1FC01EA5AFF4F0C9474
:10137000942A8C2F807FCF70882311F0C295C07F74
:10138000112399F0CC2309F4AAC180E28D0F883093
:1013900010F0D11104C08C2F0E94691103C08C2F52
:1013A0000E9479110E94A8119AC18D2F0E94E8080D
:1013B000CC2309F4A8C180E28D0F883038F1DD23F9
:1013C00029F18C2F0E947F1124C08C2F807FCF7039
:1013D000803211F0C295C07FDD2319F0D130A1F128
:1013E0003DC08091180382FF17C0112349F0CC2320
:1013F00029F08C2F0E9469110E94A81180E070C111
:1014000080E00E94E808CC2309F47DC18C2F0E9463
:101410006F110E94A81177C1112371F0002341F0D0
:10142000013031F40E9489118C2B0E9491116BC103
:101430000E9489118C2B1DC0002319F0013009F482
:1014400062C10E949E1125C0112321F0063008F0D0
:101450005AC10EC0053008F056C11BC0112361F0FF
:10146000002331F0F701858180FF39C18F708583BA
:101470008C2F0E94700947C1002359F0D93309F01D
:101480003FC1FFEF07EE13E0F15000401040E1F7DD
:1014900035C18C2F0E94770936C18C2F8695869591
:1014A000837019F0813061F02EC1112321F08D2F4E
:1014B0009C2F937002C080E090E00E94B0202BC16E
:1014C000112321F08D2F9C2F937002C080E090E0BB
:1014D0000E94C62020C18D2F112319F00E944B18A5
:1014E00002C00E94A6180E941D1915C18C2F83707E
:1014F00009F047C011110BC12D2F22952695277099
:10150000220F220F6D2F6F70862F90E0A0E0B0E0C9
:10151000022E04C0880F991FAA1FBB1F0A94D2F77E
:10152000D4FF10C04FE050E060E070E004C0440F12
:10153000551F661F771F2A95D2F7409550956095E5
:10154000709503C040E050E0BA01C695C695C370DF
:101550008A019B01082B192B2A2B3B2BC901B801AF
:10156000C23049F058F4C13019F00E947F0CCFC04E
:101570000E946D0CCCC00E94910CC9C00E946B0CE3
:10158000C6C0112319F08C2F817001C08695882365
:1015900009F4BDC02D2F229526952770220F220F0A
:1015A0006D2F6F70862F90E0A0E0B0E0022E04C097
:1015B000880F991FAA1FBB1F0A94D2F7D4FF10C02F
:1015C0004FE050E060E070E004C0440F551F661F1C
:1015D000771F2A95D2F7409550956095709503C076
:1015E00040E050E0BA01C695C695C3708A019B01E0
:1015F000082B192B2A2B3B2BC901B801C23049F00B
:1016000058F4C13019F00E94440D81C00E94320D7F
:101610007EC00E94560D7BC00E94A50C78C0CF7082
:10162000112339F08C2F0E94CB0C8D2F0E94700952
:101630006EC08D2F0E9477098C2F0E94EC0C67C022
:10164000D23F21F128F4D03F41F0D13FC1F043C057
:10165000D33F19F1D43F79F03EC0112341F005305A
:1016600008F051C08C2F8F710E94110D4CC00630B4
:1016700008F049C0F7CF8091180382FF18C01123EA
:1016800039F08C2F8F710E94CB0C3DC01123C9F310
:101690008C2F8F710E94EC0C36C0112329F08C2FF7
:1016A0008F710E94B60C2FC00E94B10C2CC0112368
:1016B00049F0CF718C2F0E94CB0C63E08C2F0E94DD
:1016C000ED1121C081E00E9408120230E0F082E0BA
:1016D0000E94081218C0112331F0002391F28D2FBF
:1016E0000E94390810C0002399F2D93349F41FEF42
:1016F00027EE33E0115020403040E1F700C00000F9
:101700008D2F0E94E80888EF8C0D843020F40E9411
:1017100041200E94A707DD20C9F00E945B1180FDD7
:1017200015C0F70112820E9455110E94CB0CC7010F
:101730000E94C70B0E945511DF91CF911F910F910D
:10174000FF90EF90DF90CF900C94EC0CDF91CF9155
:101750001F910F91FF90EF90DF90CF9008950F931E
:101760001F93CF93DF93EC01688179818A810E9476
:101770000D0E8C010E94680D0E94590CB801CE011B
:101780000E947E09DF91CF911F910F910895CF9311
:10179000DF93EC01988189812B813C81232B31F0EF
:1017A0008F3F31F481E09F3F19F403C081E001C015
:1017B00080E080FD1DC0CE010E941607811110C07F
:1017C0000E945F118823A1F08A81882389F080918B
:1017D000180382FD0DC082E0DF91CF910C940812B6
:1017E000CE010E94AF0BCE01DF91CF910C94F70692
:1017F000DF91CF91089580E090E00E94B02080E0DA
:1018000090E00E94C6200E9486110E94A8110E94AA
:10181000D01A0C941D1980910201909103010E942D
:10182000AA210C94FB0B0E9476110C940B0C929540
:101830009F70963079F010F4925001C09A50923017
:1018400068F4803F69F018F4883E40F409C0843F92
:1018500029F406C0883E20F0813F11F080E0089511
:1018600081E00895FC01808191810E94020E0E9416
:10187000170C0895CF93DF9300D000D01F92CDB7FF
:10188000DEB70F900F900F900F900F90DF91CF91D8
:101890000895CF93DF9300D000D000D0CDB7DEB74E
:1018A00026960FB6F894DEBF0FBECDBFDF91CF9165
:1018B0000895089508950C945A0C0C945B0C0E94A2
:1018C0005D0C6093390270933A0280933B029093CF
:1018D0003C020C94FB0B0C945F0C0F931F93009134
:1018E000390210913A0220913B0230913C02602B68
:1018F000712B822B932B1F910F910C945F0C0F93E4
:101900001F930091390210913A0220913B023091CD
:101910003C0260237123822393231F910F910C9427
:101920005F0C0F931F930091390210913A0220919E
:101930003B0230913C0260277127822793271F9139
:101940000F910C945F0C0C945A0C0E94A30C6093A2
:1019500035027093360280933702909338020C94CC
:10196000FB0B60E070E0CB010C94A50C0F931F9370
:1019700041E050E060E070E08A019B0104C0000F8C
:10198000111F221F331F8A95D2F7C901B8011F9179
:101990000F910C94A50C0F931F9341E050E060E071
:1019A00070E004C0440F551F661F771F8A95D2F759
:1019B0008091350290913602A0913702B0913802A1
:1019C0008A019B01082B192B2A2B3B2BC901B8013B
:1019D0001F910F910C94A50C0F931F9341E050E0C1
:1019E00060E070E004C0440F551F661F771F8A95A2
:1019F000D2F7409550956095709580913502909101
:101A00003602A0913702B09138028A019B01082367
:101A100019232A233B23C901B8011F910F910C946C
:101A2000A50C0F931F9341E050E060E070E004C00C
:101A3000440F551F661F771F8A95D2F78091350294
:101A400090913602A0913702B09138028A019B0131
:101A5000082719272A273B27C901B8011F910F9191
:101A60000C94A50C0F931F93009135021091360230
:101A70002091370230913802602B712B822B932BEF
:101A80001F910F910C94A50C0F931F930091350299
:101A90001091360220913702309138026023712371
:101AA000822393231F910F910C94A50C0F931F93E6
:101AB00000913502109136022091370230913802A0
:101AC00060277127822793271F910F910C94A50CF3
:101AD000089528E0929F800D1124E82FE695E69561
:101AE000E695877051E001C0550F8A95EAF785E0C9
:101AF000E89FF0011124E250FE4F20E030E070E05A
:101B00004081CB01022E02C0969587950A94E2F798
:101B10008170819584278523842781932F5F3F4F90
:101B20002530310569F7089528E0929F800D112432
:101B3000682F669566956695982F977085E0689FE3
:101B4000B001112440E050E080E0FB01E40FF51FFC
:101B5000E250FE4F208130E0092E02C036952795D5
:101B60000A94E2F721703327042E01C0220F0A9451
:101B7000EAF7822B4F5F5F4F4530510531F70895EB
:101B8000BF92CF92DF92EF92FF920F931F93CF936A
:101B9000DF938C01C0903502D0903602E09037027E
:101BA000F09038028091390290913A02A0913B0264
:101BB000B0913C02C82AD92AEA2AFB2ACFE1D0E018
:101BC000D701C6010C2E04C0B695A79597958795A9
:101BD0000A94D2F780FD04C0219790F7B12C07C07A
:101BE000BC2EB8018C2F0E9415150197A9F38B2DDF
:101BF000DF91CF911F910F91FF90EF90DF90CF90E9
:101C0000BF900895CF93DF93EC010E94C00DBE01F9
:101C10000E941515DF91CF9108951F93CF93DF9305
:101C2000EB019091FD01992321F0CB010E94020E5E
:101C300013C0882349F0CB010E94C00D182F682FD4
:101C4000CE010E94690D04C0CB010E94940D182F93
:101C5000BE01812F0E941515DF91CF911F9108952C
:101C60001F93CF93DF93C0913D0216E080913E0217
:101C7000C81799F0D0E01C9FF0011D9FF00D1124B2
:101C8000E15CFD4F40815181628173818481958146
:101C90000E94490C2196C770E9CFDF91CF911F9127
:101CA000089540916F02509170026091710270919D
:101CB000720280917302909174020C94490CEF921D
:101CC000FF920F931F93CF93DF93809174028295BD
:101CD0008F7009F065C080917102882309F460C09B
:101CE00080913D02F0903E0210916F0200917002CF
:101CF000609172027091730291E01F3F09F090E0D1
:101D0000C0910001D0910101292F96E0E92E8F1595
:101D100009F446C06115710521F00F3F21F030E054
:101D200003C031E001C0322F90E030FD36C0E89EA4
:101D3000F001E99EF00D1124DF01A15CBD4F119669
:101D40003C911197301329C03C91311326C0129653
:101D50003C911297311121C013964D915C911497CB
:101D6000461B570B4C175D07C0F4809174028F70AF
:101D7000806180937402EC5BFD4F80818F70806185
:101D800080838FE692E00E94C70BDF91CF911F9175
:101D90000F91FF90EF900C94300E01968770B7CFA3
:101DA000DF91CF911F910F91FF90EF9008959F9237
:101DB000AF92BF92CF92DF92EF92FF920F931F9359
:101DC000CF93DF93CDB7DEB761970FB6F894DEBF40
:101DD0000FBECDBF8C0185E0F801DE011D9601909C
:101DE0000D928A95E1F7D8011296EC9090916F02CE
:101DF000E091700220917202309173022115310539
:101E000031F0EF3F31F481E09F3F19F403C081E0EE
:101E100001C080E0B82FB1709B2E80FD47C1D80172
:101E20004C9111965C9111971396AD90BC901497BC
:101E30008FE6C82E82E0D82EF0907102B501621BA9
:101E4000730B2091000130910101FF2009F4D9C0EA
:101E5000809174026217730708F095C0282F207FC5
:101E600009F052C05E1313C0491311C0FE2CE110DB
:101E70000EC08F708061809374020E94510EC60163
:101E80000E94C70B80917402F80185834DC1AB2875
:101E900031F05F3F31F481E04F3F19F403C081E03E
:101EA00001C080E080FD03C081E08E2502C080E09B
:101EB00090E0F82FF170FF2E80FF1CC080913D0252
:101EC00020913E0236E0821709F40BC190E0389F62
:101ED000F001399FF00D1124E15CFD4F6181561333
:101EE00006C06081461303C06281E61203C00196FA
:101EF0008770E9CFFE2CEE2009F416C180917402A0
:101F000081608093740254C05E1306C0491304C0FC
:101F1000E11002C0F80199C0C8010E94320C882368
:101F200061F1EE2051F120917402822F82958F7021
:101F300090E0029774F080916F0290917002988700
:101F40008F831986BB86AA862C87CE0107960E94AE
:101F5000C70B86E0F801AFE6B2E001900D928A95DA
:101F6000E1F70E945F0E0E94510E0AC05E1711F148
:101F7000C8010E94320C81112CC0C8010E94C70BFD
:101F8000FF24F394D1C0282F207F81F77A2DB98ABE
:101F9000A88A6E2D89890E943A0C8FE692E00E94F1
:101FA000C70B86E0D6011D928A95E9F70E94510E73
:101FB000F12CBAC04913DCCFE110DACFF8018583E8
:101FC000C8010E94C70B86E0D6011D928A95E9F7E9
:101FD000ABC0EE2091F220917402822F82958F7017
:101FE00090E002970CF4B5CF80916F02909170024F
:101FF0009A8389831B82BD82AC822E83CE01019697
:10200000A6CF6217730708F044C0FE2CEE2009F437
:10201000B4CF5E1330C049132EC02091740220FD4E
:1020200021C0822F82958F70482F50E041155105B5
:10203000C9F0F80125834F30510541F08F5F982F8B
:102040009295907F822F8F70892B8583C8010E9483
:10205000C70B86E0F801AFE6B2E001900D928A95D9
:10206000E1F73CC086E0F801AFE6B2E001900D92E6
:102070008A95E1F759C0C8010E94320C811169CFDD
:1020800080917402816080937402C8010E94C70B22
:102090004BC07A2DB98AA88A6E2D89890E943A0C84
:1020A00086E0D6011D928A95E9F718C0EE2009F462
:1020B00064CFC8010E94320CF82E882309F45DCF4A
:1020C00086E0F801AFE6B2E001900D928A95E1F763
:1020D0008FE692E00E9433080E945F0E0E94510E2C
:1020E00023C04D875E878D859E850E94020E292F15
:1020F00022952F70223028F49F7039F0811105C08D
:102100000BC0243028F49F7049F4805E883020F0A2
:10211000C8010E94C70B9F2CF92C06C0D801159648
:102120009C91907F91F7F8CF8F2D61960FB6F89420
:10213000DEBF0FBECDBFDF91CF911F910F91FF90FA
:10214000EF90DF90CF90BF90AF909F9008951F9336
:10215000CF93DF93CDB7DEB72C970FB6F894DEBFE1
:102160000FBECDBF4F83588769877A878B879C873F
:10217000CE0107960E94D70E8823D1F09F818885D3
:102180002A853B85232B31F08F3F31F481E09F3F3F
:1021900019F403C081E001C080E080FD47C04F8199
:1021A000588569857A858B859C850E94490C3EC03F
:1021B00086E0FE013796DE01119601900D928A9518
:1021C000E1F7FF81E8856A857B856115710531F04E
:1021D000EF3F31F481E0FF3F19F403C081E001C01B
:1021E00080E080FD23C020913E0230E0C9010196CD
:1021F0008770992740913D0250E084179507F1F1CF
:10220000F983EA837D836C8396E0929FD001939F4C
:10221000B00D1124A15CBD4FFE01319601900D92CD
:102220009A95E1F780933E020E94300E16E080916D
:102230003D0290913E02891771F1189FC00111244F
:10224000815C9D4F0E94D70E882329F1E0913D02C9
:102250001E9FF0011124E15CFD4F4081518162819C
:102260007381848195810E94490C80913D0290E0A8
:1022700001968770992780933D02D9CF0E94130C55
:1022800010923E0210923D02EFE6F2E086E0DF019E
:102290001D928A95E9F72C960FB6F894DEBF0FBE13
:1022A000CDBFDF91CF911F910895809195028595C3
:1022B00085958595089580919502877008959091F0
:1022C0009502977081E009F480E008958091B8024A
:1022D00008959091B802892B8093B8020895809553
:1022E0009091B80289238093B80208951092B802A1
:1022F00008959091B702892B8093B7020895809535
:102300009091B70289238093B70208951092B70283
:10231000089580919602089508950C948C110C9460
:102320008D119091180392FD08C090919602981714
:1023300021F0809396020C948F110895809196025B
:10234000882329F01092960280E00C948F11089552
:10235000CF93DF93E0910201F09103018091B802E5
:102360008083E0910201F091030190818091B70296
:10237000892B808380919602882381F0E09102016D
:10238000F09103019081892B8083809102019091CB
:1023900003010E94DC2081110E949E11C091020164
:1023A000D091030140E250E065E772E0CE010E9467
:1023B000AE2A892B69F080E2FE01A5E7B2E0019028
:1023C0000D928A95E1F7CE01DF91CF910C944D20CB
:1023D000DF91CF9108950C948C119091180392FD88
:1023E00010C098E0899F90011124262B209395021C
:1023F0000E94CB0C809195028595859585950C94CE
:10240000EB110C94CB0C1092950280E00C94EB1124
:10241000209195028095822380939502982F977042
:1024200099F430E0482F082E000C550B241735077F
:1024300059F09091180392FD07C085958595859573
:102440000E94EC0C0C9403120895CF939091180302
:1024500092FB222720F92817F9F0C82F892FC0FBFB
:1024600082F98093180380911703909118030E94BA
:10247000871282E00E9408128091CC0280FF0CC07B
:102480001F92CF938BE392E09F938F930E948F06CE
:102490000F900F900F900F90CF9108958091180397
:1024A00082FB882780F991E089270C94251281E02E
:1024B0000C94251280E00C9425126FEF7FEF80E0E2
:1024C00090E00C94E72A80E090E00E94C32A21E08B
:1024D000893E9E4F09F020E0822F089582E090E02F
:1024E0000C94BB2A83E090E00C94BB2ACF9384E049
:1024F00090E00E94BB2AC82F82E290E00E94BB2A93
:102500002C2F30E0A901582BCA01CF910895CF9309
:10251000C92F682F84E090E00E94C92A6C2F82E2C4
:1025200090E0CF910C94C92AAB01BC018FE090E000
:102530000C94DB2AAB01BC0183E190E00C94DB2A14
:1025400060E070E0CB010C949A1260E070E0CB0187
:102550000E9494120C94A01269EE7EEF80E090E04D
:102560000E94E72A60E082E090E00E94C92A60E0D1
:1025700083E090E00E94C92A1092390210923A0238
:1025800010923B0210923C0260E084E090E00E94D6
:10259000C92A60E082E290E00E94C92A60E085E0FA
:1025A00090E00E94C92A60E086E090E00E94C92A7B
:1025B0006FEF87E090E00E94C92A40E050E0BA0146
:1025C00088E090E00E94DB2A60E08DE090E00E94CD
:1025D000C92A40E050E0BA0188E190E00E94DB2A7D
:1025E00060E087E190E00E94C92A40E050E0BA0133
:1025F0008CE190E00E94DB2A60E070E080E290E0F5
:102600000E94E72A40E050E0BA0188E190E00E9491
:10261000DB2A0C94A5120C94AC12682F8EE090E08B
:102620000C94C92A0E9463226093C8027093C90265
:102630008093CA029093CB026093C4027093C50248
:102640008093C6029093C702089585B7806885BFBE
:1026500085B7806885BF089581E008950C942C1398
:1026600008950C9430130C9430130C9433130C9481
:1026700030130C9437130C9430130E9425138EEBF7
:1026800094E20E9437200E943B130C9439130E945D
:1026900031130C9430130E9409160C94A6070E9463
:1026A0004E220E9423170E944B13E7E1F3E0808142
:1026B0008068808380911703909118030E9487128D
:1026C0000C9435138F929F92AF92BF92CF92DF926C
:1026D000EF92FF920F931F93CF93DF93CDB7DEB7A7
:1026E0002A970FB6F894DEBF0FBECDBF0E943817F1
:1026F000982E81110E94121389EBA82E82E0B82E29
:1027000000E010E0802E802F0E942D16D82EF501BB
:10271000C1905F01C826B1F40F5F1F4F0B30110548
:1027200089F78FEF89838A831B820E9457228160F9
:10273000782F9D838C8349815A816B818D810E9482
:10274000E9072FC08091CC0281FD0E943316E12C55
:10275000FF24F3948C2D8F21F1F00E942E138823F7
:1027600099F0EE828F82DF2081E009F480E0888793
:102770000E9457228160782F9A8789874E815F81D6
:1027800068858A850E94E907F801E754FD4F80813A
:10279000F826F08206C0E394FF0CF8E0EF12DACFDF
:1027A000BBCF81E0911001C080E02A960FB6F8946B
:1027B000DEBF0FBECDBFDF91CF911F910F91FF9074
:1027C000EF90DF90CF90BF90AF909F908F90089543
:1027D0000E9462130E94BD190C94B707CF93DF9338
:1027E0000E941A15EC01811521E5920708F045C0F9
:1027F000811530E5930708F094C0883E910528F5CF
:10280000803E910508F0F8C0883A910570F4853A49
:10281000910508F07CC08130910509F475C008F479
:10282000E8C0049708F0E8C0E4C08F3B910508F0C9
:10283000E0C0C85AD0E0CC0FDD1FC65BDE4F099068
:10284000D881C02DCE019464D8C0811540E2940790
:1028500058F4811551E0950708F0CEC08D3E9105E2
:1028600008F4C7C09065C9C0C11580E4D80708F452
:10287000C0C0DF70CE01906AC0C0811525E5920707
:10288000A8F4811534E5930708F095C0811543E558
:10289000940708F07BC0811552E5950708F061C0E8
:1028A000D82FCC27CE01816F906AA7C0C11589E5CA
:1028B000D807A0F4C11528E5D20708F082C0C115D9
:1028C00036E5D30708F095C08C2F0E94AE158F71A6
:1028D00090E0D82FCC27CE0190628FC0C1154AE579
:1028E000D40708F474C0CE0190568115904208F0C8
:1028F00080C08D2F8F710E94AE15DD27D0628F7141
:10290000AE01582BCA0179C081E090E076C0C55A6B
:10291000D0E0C858DE4F8881C82FD0E0CE01906447
:102920006CC074E0969587957A95E1F7282F23700F
:102930003C2F337081E090E002C0880F991F3A95D8
:10294000E2F79C68AC01522B9A019C2F9F709695E0
:10295000969550E2959FE0011124C9018C2B9D2B87
:102960004CC08370992721E030E002C0220F331F52
:102970008A95E2F79C2F9695969580E2989FE001C4
:102980001124C22BD32BCE019C6837C083709927AA
:1029900021E030E002C0220F331F8A95E2F79C2F1E
:1029A0009695969540E2949FE0011124C22BD32B7B
:1029B000CE019A6822C0D82FCC27CE01846F906AAE
:1029C0001CC0DC2FCC27CE01806F906A16C08C2FE4
:1029D0008F700E94AE1594E0D695C7959A95E1F751
:1029E000CF70D0E0DC2FCC27D0699E01282BC90105
:1029F00004C080E090E001C0CE01DF91CF91089546
:102A0000E72FF0E09BE0899FE00DF11D112483E0AA
:102A1000EE0FFF1F8A95E1F7E60FF11DEE0FFF1F86
:102A2000EA5AFE4F8591949108950E9400150E94E4
:102A3000EE1308958238910569F1B0F48133910560
:102A400009F46DC048F48932910509F463C08A32F3
:102A5000910509F469C008958533910509F455C0BD
:102A600089339105B9F00895833E910569F138F4F1
:102A7000803E9105B1F0823E910509F10895863EB0
:102A80009105A9F1873E9105B9F1843E910509F0C0
:102A900064C023C02091170320FD4FC021FD4DC00D
:102AA00008958091170380FD44C08091180380FF32
:102AB00044C08091170384FD42C083EE4DC08091D5
:102AC000170382FF38C0F5CF8091170382FD33C012
:102AD0008091180380FD31C0ECCF8091180381FFF5
:102AE00032C08091170384FD2AC087EE35C08091E3
:102AF000170383FF26C0F5CF8091170383FD21C004
:102B00008091180381FD1FC0ECCF8091170385FDD4
:102B10001CC01DC08091170385FD19C016C080918F
:102B2000170386FD16C017C08091170386FD13C0DA
:102B300010C089E311C082EE0FC080EE0DC080E0AE
:102B40000BC086EE09C084EE07C089E205C085E3AC
:102B500003C08AE201C081E390E0089590911703D9
:102B600092FF0DC0282F2871283019F4877F8460C8
:102B700006C0282F2471243011F48B7F886093FFC6
:102B80000DC0282F2871283119F4877E846106C072
:102B9000282F2471243111F48B7E88612091180331
:102BA00020FF0DC0382F3871383019F4877F8160CD
:102BB00006C0382F3171313011F48E7F886021FFCB
:102BC0000DC0282F2871283119F4877E816106C035
:102BD000282F2171213111F48E7E886194FD877E2A
:102BE00008950C945D120E9438178FE39CE90197B9
:102BF000F1F700C000000E94381780E00E942D16F7
:102C000080FF04C00E94F1150C94A42208950C9436
:102C1000F3150E946312811102C00E940B130E94DF
:102C20006E128093CC020E947612909318038093C8
:102C300017030E9407160E947212682F70E080E04E
:102C400090E00E946B0C6091350270913602809189
:102C50003702909138020C94A30CE82FF0E0EC5D61
:102C6000FC4F80810895CF92DF92EF92FF920F93F5
:102C70001F93CF93DF938FE592E00E94F60584E2E5
:102C8000E82E83E0F82EC0E0D0E09AE5C92E92E06D
:102C9000D92E02E512E0DF93CF93DF92CF920E940C
:102CA0008F0687E592E00E94F605F70181917F018A
:102CB0000E948F071F928F931F930F930E948F067E
:102CC00080E592E00E94F60521968DB79EB70896A2
:102CD0000FB6F8949EBF0FBE8DBFCB30D105D9F68D
:102CE000DF91CF911F910F91FF90EF90DF90CF90E8
:102CF000089580EA8A95F1F7089500C008950C942C
:102D0000791608950C9481160C9482160C948116F1
:102D1000F894E82FE295EF70F0E031A1282F2F70A2
:102D200081E090E001C0880F2A95EAF7982F9095EE
:102D3000932391A392A1892B82A3789408950F9352
:102D40001F93CF93DF93C3E8D1E089918F3F11F0B8
:102D50000E94881681E0CE38D807B9F7CBE7D1E0DA
:102D600003E811E089918F3F11F00E9488160C173B
:102D70001D07C1F7DF91CF911F910F910895CF9259
:102D8000DF92EF92FF920F931F93CF93DF938C010B
:102D9000C62FD0E0CE018D579E4F7C01FC01908163
:102DA0009F3F09F447C0D62EF894E92FE295EF70C3
:102DB000F0E081A19F7021E030E001C0220F9A95E0
:102DC000EAF7822B81A382A12095282322A378945D
:102DD0000E947D16EBE7F1E043E851E031E0C12CC1
:102DE00021912F3F89F0A22FA295AF70B0E090966D
:102DF0008C9190E02F7002C0959587952A95E2F707
:102E000080FD02C0832F01C080E0C82A330F4E1717
:102E10005F0731F7F70180818F3F11F00E9488161C
:102E200061E0C11001C060E08D2D0E947F16C00FCF
:102E3000D11FC882DF91CF911F910F91FF90EF902A
:102E4000DF90CF9008950E949F168BE0E4E2F3E0BC
:102E5000DF01982F1D929A95E9F7E9E1F3E0DF0190
:102E60001D928A95E9F78BE00E9483170C94020764
:102E7000FF920F931F93CF93DF93CDB7DEB72B97BE
:102E80000FB6F894DEBF0FBECDBF8E010F5F1F4F90
:102E90008BE0F80111928A95E9F7F12C6F2DC801AA
:102EA0000E94BF16F394FBE0FF12F8CF4BE050E016
:102EB000B80189E193E00E94AE2AFF24F3940097C1
:102EC00009F4F12C892B41F08BE0F801A9E1B3E082
:102ED00001900D928A95E1F72F2D4BE064E273E0AB
:102EE00089E193E00E9484170E9404078F2D2B969E
:102EF0000FB6F894DEBF0FBECDBFDF91CF911F910B
:102F00000F91FF9008950895FF920F931F93CF9311
:102F1000DF938C01F62ED72FC42F222349F081E0B6
:102F20008093CF020E9457229093CE028093CD02CD
:102F30008091CF028823C1F08091CD029091CE0282
:102F40000E946F22059780F0EF2DFD2FD8014C2FA6
:102F500050E0CD01801B910B841795071CF48D91D7
:102F60008193F7CF1092CF02DF91CF911F910F91F4
:102F7000FF9008950E943A250E944F130C94462515
:102F80000E944A250E94E8130C9468250E94F521AE
:102F90000E9421250E943D130E94BA170E94C0176B
:102FA0000E944713FBCF8091D60280FF06C060913C
:102FB000090170E0660F771F26C081FF04C0609191
:102FC000090184E005C082FF07C06091090188E023
:102FD000689FB001112417C09091D5029923D1F0B8
:102FE00060910801961788F72091090188E0289FD1
:102FF00090011124929FA001939F500D112470E025
:10300000CA010E94802A6038710540F4611571057B
:1030100019F406C068E070E0862F08958FE70895E0
:1030200081E008958091D60280FF08C0609105017B
:1030300070E0759567957595679521C081FF06C00D
:103040006091050170E07595679519C082FF04C015
:103050006091050170E010C09091D402992399F01D
:10306000609104019617A0F780910501899FC00126
:10307000112470E00E94802A6038710540F46115C7
:10308000710519F406C061E070E0862F08958FE79E
:10309000089581E008958D3E21F40E94D317819513
:1030A00004C08E3E29F40E94D3178093DA0208955B
:1030B0008F3E21F40E94D317819504C0803F29F4EC
:1030C0000E94D3178093D9020895893F19F40E9472
:1030D000121805C08A3F31F40E941218819580931E
:1030E000DB0208958B3F21F40E941218819504C0E1
:1030F0008C3F29F40E9412188093DC0208959FE00F
:10310000980F983078F421E030E0A90102C0440F14
:10311000551F9A95E2F7CA019091D802892B8093A6
:10312000D80208958D3F21F48091D60281600BC0B2
:103130008E3F21F48091D602826005C08F3F29F432
:103140008091D60284608093D60208958D3E39F432
:103150009091DA0297FF35C01092DA0259C08E3E84
:1031600029F49091DA021916BCF32BC09091D90280
:103170008F3E29F497FF25C01092D90249C0803FA5
:1031800019F41916CCF31DC09091DB02893F29F484
:103190001916BCF41092DB023BC08A3F19F497FF6A
:1031A00010C0F8CF8B3F39F49091DC0297FF09C033
:1031B0001092DC022DC08C3F21F49091DC02191694
:1031C000BCF39FE0980F983080F421E030E0A90133
:1031D00002C0440F551F9A95E2F7CA01809590915D
:1031E000D80289238093D80213C08D3F21F48091A7
:1031F000D6028E7F0BC08E3F21F48091D6028D7F48
:1032000005C08F3F29F48091D6028B7F8093D60230
:103210008091D902811106C08091DA02811102C029
:103220001092D5028091DB02811106C08091DC02F0
:10323000811102C01092D40208958091CC0283FFC4
:103240007EC085E992E00E94F6058091D8021F9227
:103250008F9380E992E09F938F930E948F068EE870
:1032600092E00E94F6058091D902282F082E000CCA
:10327000330B3F938F938BE892E09F938F930E9441
:103280008F0689E892E00E94F6058091DA02282FE5
:10329000082E000C330B3F938F9386E892E09F93A8
:1032A0008F930E948F0684E892E00E94F605809139
:1032B000DB02282F082E000C330B3F938F9381E8FD
:1032C00092E09F938F930E948F068FE792E00E9477
:1032D000F6058091DC02282F082E000C330B3F935B
:1032E0008F938CE792E09F938F930E948F0689E7DC
:1032F00092E00E94F6058091D5021F928F9386E797
:1033000092E09F938F930E948F0684E792E00E9441
:10331000F6058091D6021F928F9381E792E09F93EA
:103320008F930E948F068EE692E00E94F6058DB77D
:103330009EB74C960FB6F8949EBF0FBE8DBF0E94ED
:1033400057222091D902211104C02091DA022223B0
:1033500021F09093D3028093D2022091DB022111BD
:1033600004C02091DC02222321F09093D1028093AB
:10337000D00287ED92E00C94A220EF92FF920F937F
:103380001F93CF93DF9300D000D000D0CDB7DEB72E
:1033900086E0E7EDF2E0DE01119601900D928A954C
:1033A000E1F7E090D902F090DA020091DB0210918F
:1033B000DC021092D9021092DA021092DB02109213
:1033C000DC02E11003C0FF2009F45DC08091D2024D
:1033D0009091D3020E946F22AC019091D502992363
:1033E00039F020910A0130E02417350758F04BC01E
:1033F00020910B018AE0289F9001112424173507A2
:1034000018F041C09F3F19F09F5F9093D502EE20C6
:1034100061F00E94D3171E1414F09FEF01C091E0D9
:10342000989F902D11249093D902FF2061F00E9463
:10343000D3171F1414F09FEF01C091E0989F902DB7
:1034400011249093DA023091D9023323E1F02091D4
:10345000DA022223C1F045EB3403C0011124992381
:1034600019F09093D90203C081E08093D90235EB23
:103470002303C0011124992319F09093DA0203C0A9
:1034800081E08093DA02011103C0112309F45DC0C9
:103490008091D0029091D1020E946F22AC01909154
:1034A000D402992339F02091060130E02417350722
:1034B00058F04BC0209107018AE0289F9001112409
:1034C0002417350718F041C09F3F19F09F5F909374
:1034D000D402002361F00E941218101614F09FEF1E
:1034E00001C091E0989F902D11249093DB0211234D
:1034F00061F00E941218111614F09FEF01C091E0C4
:10350000989F902D11249093DC023091DB0233239D
:10351000E1F02091DC022223C1F045EB3403C0012D
:103520001124992319F09093DB0203C081E080936A
:10353000DB0235EB2303C0011124992319F090938A
:10354000DC0203C081E08093DC028091D90281110A
:103550000BC08091DA02811107C08091DB028111DA
:1035600003C08091DC0281110E941D19EB82FC8254
:103570000D831E8386E0FE013196A7EDB2E0019037
:103580000D928A95E1F726960FB6F894DEBF0FBE2E
:10359000CDBFDF91CF911F910F91FF90EF900895D4
:1035A000E7EDF2E086E0DF011D928A95E9F71092DF
:1035B000D5021092D4021092D6020895CF93DF93D1
:1035C000EC01FB018281882309F43CC1C430FDE594
:1035D000DF0760F4CB3F9CE5D90788F49E012250B9
:1035E0003C452431310508F02EC109C0C236EDE555
:1035F000DE0729F0C63AFDE5DF0709F024C10E9485
:1036000076129093180380931703C1318CE5D80785
:1036100009F4C6C008F042C0C930ECE5DE0709F481
:103620009BC000F5C5308CE5D80709F485C078F457
:10363000C330ECE5DE0709F478C008F07AC0C23088
:10364000DC4509F0F5C0809117038160EFC0C730F9
:103650009CE5D90709F478C008F07AC08091170377
:103660008061E4C0CD30FCE5DF0709F487C058F481
:10367000CB309CE5D90709F479C008F07BC0809174
:10368000170388606FC0CF30FCE5DF0709F480C006
:1036900008F082C080911703877FC8C0CE3F9CE5A9
:1036A000D90709F471C000F5C531FCE5DF0709F45D
:1036B00085C068F4C3319CE5D90709F475C008F0EA
:1036C00095C00E94130C809117038F77AFC0CC3F39
:1036D000FCE5DF07A9F108F054C0CB3FDC4509F059
:1036E000A7C08091180340C0C230EDE5DE0709F4A1
:1036F00089C058F4C1158DE5D80709F45AC008F0FF
:1037000069C08091180382602FC0C236EDE5DE07E4
:1037100009F47CC0C63AFDE5DF0709F481C0C33077
:10372000DD4509F085C080E06EC08091170382609E
:103730007DC08091170316C080911703886076C002
:103740008091180382604FC08091170380626EC021
:103750008091170380646AC00E94130C8091170344
:10376000806864C0846062C081603DC0809117033E
:103770008E7F5CC0809117038D7F58C080911703A6
:1037800016C08091180318C0809118038D7F2BC03C
:10379000809117038F7E4AC0809117038F7D46C0AA
:1037A000809117038F7B42C080911703877F8B7FA7
:1037B0003DC0809118038D7F8E7F15C080911703C7
:1037C00082FB222720F991E0922790FB82F990FB5F
:1037D00083F92CC080911803982F909591708E7F5B
:1037E000892B90FB81F98093180322C00E94130C4F
:1037F0008091170387FB222720F991E0922790FB05
:1038000087F914C081E00E940D1312C08091170344
:1038100084FB222720F991E0922790FB84F906C0CF
:1038200080911703982F909590FB80F98093170350
:1038300080911703909118030E9487120E94130C25
:1038400080E001C081E0DF91CF9108958091040173
:103850001F928F93809105011F928F938091080191
:103860001F928F93809109011F928F9380910A017B
:103870001F928F9380910B011F928F9388EB92E0A0
:103880009F938F930E948F068DB79EB70E960FB6AB
:10389000F8949EBF0FBE8DBF0895883220F58E31FB
:1038A00008F068C08B3091F1C0F4873009F0BEC0D9
:1038B00081E080930B0184E180930A018AE0809388
:1038C00009018EE18093080188E08093050188E278
:1038D000809304018AE194E0C6C0833109F443C0B7
:1038E000843169F1A3C08F3409F49EC028F4893271
:1038F00031F1883359F09AC0813531F008F4D4C0E1
:10390000823509F4A7C092C08FEFA5C08CE394E084
:103910000E94F6050E94261C1F9281E08F931F9241
:1039200088E08F9385E393E09F938F930E948F06A7
:103930000F900F900F900F900F900F9096C089E30B
:1039400094E00E94F6058091E102882309F4AAC060
:103950001092E1021092E0021092DF021092DE0259
:103960001092DD02B1C08BE294E00E94F6050E9445
:10397000261C7BC08D518093E102833031F170F4BD
:103980008130D1F0823009F03FC08AE091E090931D
:10399000E0028093DF028BE991E01FC0853059F18E
:1039A00008F1863089F584E091E09093E0028093FD
:1039B000DF0286ED91E011C08BE091E09093E00290
:1039C0008093DF0282E991E008C089E091E0909362
:1039D000E0028093DF0287EA91E09093DE02809319
:1039E000DD0218C088E091E09093E0028093DF024E
:1039F00084EB91E0F2CF85E091E09093E002809338
:103A0000DF0283EC91E0E9CF1092E10288E294E0DA
:103A10000E94F6058091E102882309F455C01F92A7
:103A20008F9384E294E00DC08AE015C087E194E0B2
:103A30001AC097FF47C0108280811F928F9381E147
:103A400094E09F938F930E948F060F900F900F909A
:103A50000F900BC081E0E091DF02F091E00230971F
:103A600029F58EE094E00E94F6052091E1022223E0
:103A700059F18091DD029091DE02009711F48EE8F9
:103A800091E09F938F931F922F9385E094E09F93F3
:103A90008F930E948F060F900F900F900F900F90B2
:103AA0000F9016C080E0089586EFD5CF2081082EB4
:103AB000000C990B820F911D8F3F910509F00CF4BA
:103AC000B8CF8FEF8083B8CF81E094E00E94F605F5
:103AD00081E00895CF93C82F1F928F9382E594E0E1
:103AE0009F938F930E948F0681E090E0A0E0B0E06A
:103AF000BC01CD0104C0660F771F881F991FCA95AE
:103B0000D2F70E946B0C0F900F900F900F90CF91F7
:103B10000C94130CDF92EF92FF920F931F93CF93AD
:103B2000DF93482F50E0FA013597EF33F10508F0A5
:103B30003FC1EE59FF4F0C94942A0E9472121F92BB
:103B40008F9383EA98E09F938F930E948F060E9441
:103B50006E1283FB992790F91F929F9382FB9927FE
:103B600090F91F929F9381FB992790F91F929F9341
:103B7000982F91701F929F931F928F938AE598E0E0
:103B80009F938F930E948F060E94761287FB2227B5
:103B900020F91F922F9386FB222720F91F922F9343
:103BA00085FB222720F91F922F9384FB222720F9DF
:103BB0001F922F9383FB222720F91F922F9382FBC2
:103BC000222720F91F922F9391FB222720F91F9281
:103BD0002F93292F21701F922F9381FB222720F9E9
:103BE0001F922F93282F21701F922F939F938F93B3
:103BF00085E797E09F938F930E948F068DB79EB7BE
:103C000088960FB6F8949EBF0FBE8DBF06C083E6A0
:103C100099E00E94F6050E940B13C1E0CEC083EC30
:103C200095E074C08091CC02817F8E7F8093CC021E
:103C30008CE995E00E94F6058FE599E00E94F60573
:103C400081E08093E202E9CF83E499E00E94F605E7
:103C50000E940707E2CF8091CC02C82FC095C170A7
:103C6000C0FB80F98093CC02CC2319F087E399E064
:103C700091C08AE299E00E94F6058091CC02897F8A
:103C8000877F8093CC02C9CF9091CC0291FBCC2747
:103C9000C0F981E0C827892FC0FB81F98093CC024D
:103CA000CC2319F08DE199E027C08FE099E02EC078
:103CB0009091CC0292FBCC27C0F981E0C827892FD4
:103CC000C0FB82F98093CC02CC2319F080E099E00C
:103CD00013C080EF98E01AC09091CC0293FBCC27E0
:103CE000C0F981E0C827892FC0FB83F98093CC02FB
:103CF000CC2351F084EE98E00E94F6058091CC022E
:103D000081608093CC0259C087ED98E00E94F6054F
:103D100084CF8BED94E0FACF0E946322062FF72E1A
:103D2000E82ED92EC0911703C7FBCC27C0F91091FC
:103D30001603D09118010E944120DF92EF92FF926A
:103D40000F931F92CF931F921F931F92DF931F9287
:103D50008F9387E594E09F938F930E948F068DB792
:103D60009EB70E960FB6F8949EBF0FBE8DBF55CF6F
:103D70000E94130C9091170397FBCC27C0F981E0A8
:103D8000C827892FC0FB87F980931703CC2329F01C
:103D90008DEC98E00E94F60510C082EC98E0B6CF5A
:103DA000895303C08D5101C080E00E946A1D35CF48
:103DB00080EC98E00E94F605C0E08C2FDF91CF9157
:103DC0001F910F91FF90EF90DF90089580E008958C
:103DD0000C94E61ECF93C82F8091E202813071F0DF
:103DE00040F0823009F045C08C2F0E944D1C81E0CC
:103DF00046C00E9466118232F1F504C00E9466112D
:103E0000823261F48C2F0E94E81E811104C08C2F35
:103E10000E948A1D2CC081E090E029C08C2F0E9456
:103E2000E61E811123C0C431C9F058F4CB3069F0CB
:103E3000C031B9F482E08093E20288E30E944D1C15
:103E400015C0C93259F0C83361F48CE995E00E947D
:103E5000F6058EE494E00E94F60508C01092E20296
:103E60000CC08CE494E00E94F60507C081E08170EC
:103E700006C01092E20280E002C080E0F8CFCF914D
:103E80000895CF93DF9386319C4541F5EB010E9465
:103E90006611982F8A8120910201309103018823B5
:103EA00079F09A7A81E009F480E08093E30291113D
:103EB00002C069E201C065E3C9010E9494210AC001
:103EC0008091E302811102C069E201C065E3C9018A
:103ED0000E949F210E94A81180E001C081E0DF9133
:103EE000CF9108950F931F93CF93DF93C42FD22FB9
:103EF000FC0182818823C9F04093E6020E94572288
:103F00009093E5028093E40280E28C0F883008F001
:103F100057C0C77081E001C0880FCA95EAF7DF91EA
:103F2000CF911F910F910C9470098091E602481374
:103F300030C08091E4029091E5020E946F22883C9B
:103F4000910538F510E21D0FCD17B9F080E28C0F06
:103F5000883040F4C77081E001C0880FCA95EAF745
:103F60000E947709183028F581E09D2F977001C0D5
:103F7000880F9A95EAF70E947009802F0E946709BE
:103F80001830F0F4D77081E001C0880FDA95EAF7B5
:103F90000AC080E28C0F883098F4C77081E001C0BD
:103FA000880FCA95EAF7DF91CF911F910F910C947A
:103FB0007709802FDF91CF911F910F910C946709A2
:103FC000DF91CF911F910F9108950F939C01CB0129
:103FD000243F4CE5340731F188F4293DFCE53F07E7
:103FE000D9F02A3D4CE5340779F1283D3C45A9F547
:103FF00006E221EE41EE68ED7CE52BC0263FFCE5B4
:104000003F07E1F0A8F0273F3C4539F507E225EEF0
:1040100046EE67EF7CE51DC007E225EE45EE69ED53
:104020007CE517C006E221EE40EE64EF7CE511C0AE
:1040300007E225EE44EE65EF7CE50BC006E221EEDB
:1040400042EE66EF7CE505C008E221E045EE6AED50
:104050007CE50E94721F80E008C0FC0182818823F9
:1040600019F01092E60201C081E00F91089590933B
:10407000FB018093FA0108959093EC028093EB0288
:104080000895E091EB02F091EC02309721F001905D
:10409000F081E02D099480E00895EF92FF921F9344
:1040A000CF93DF93FC01A091EB02B091EC0210974B
:1040B00009F442C080911801882341F080911703D0
:1040C00087FF04C08081818386E08083EF011296A0
:1040D000ED91FC911397CE0109958091CC0282FF5E
:1040E0002BC080FF04C08CE799E00E94F60518E021
:1040F00086E7E82E89E0F82E8091CC0280FF0BC085
:1041000088811F928F93FF92EF920E948F060F90EB
:104110000F900F900F90115021961111EDCF8091BB
:10412000CC0280FF09C084E799E0DF91CF911F9115
:10413000FF90EF900C94F605DF91CF911F91FF90C7
:10414000EF900895E091EB02F091EC02309739F096
:1041500022E0DC012C930480F581E02D0994089580
:104160002091E9023091EA022817390771F0909303
:10417000EA028093E902E091EB02F091EC023097C1
:1041800021F00680F781E02D099408952091E7023F
:104190003091E8022817390771F09093E802809374
:1041A000E702E091EB02F091EC02309721F00084FD
:1041B000F185E02D09940895FC0132968091180153
:1041C000882331F08091170387FF02C09EE101C070
:1041D00096E080E0915028F021912223D9F38F5F5F
:1041E000F9CF0895662351F1209118012223E9F0B7
:1041F0002091170327FF19C0462F469546954695EF
:104200004E31E0F4677021E030E002C0220F331F2E
:104210006A95E2F7FC01E40FF11D828190E028230A
:10422000392381E0232B69F409C0FC0132960896FA
:104230002191621729F0E817F907D1F780E0089576
:1042400081E008959C01FC0132969FEF80E041914E
:10425000461789F09F3F19F4411101C0982F8F5FD5
:104260008630A9F79F3F39F0F901E90FF11D97FD5D
:10427000FA956283089508959C012A5F3F4FFC01DF
:104280004281461301C01282019682179307B9F743
:104290000895262F2695269526952E3170F4FC013B
:1042A000E20FF11D677021E030E001C0220F6A9536
:1042B000EAF78281282B228308958091CC0280FF27
:1042C0000CC01F926F938CEA99E09F938F930E948A
:1042D0008F060F900F900F900F900895262F269520
:1042E000269526952E3178F4FC01E20FF11D6770BA
:1042F00021E030E001C0220F6A95EAF72095828123
:104300002823228308958091CC0280FF0CC01F9245
:104310006F938EE899E09F938F930E948F060F9082
:104320000F900F900F90089520911801222329F0EB
:104330002091170327FD0C9449210C9422212091F0
:104340001801222329F02091170327FD0C946E21D8
:104350000C943C2120911801FC013296222331F06B
:104360008091170387FF02C08EE101C086E0DF0164
:104370001D928A95E9F7089508950C94BC2183E075
:104380008093ED020C94BD21811102C081E001C037
:1043900082E08093ED020C94BD210C94C42181E055
:1043A0008093ED020C94BD210C94CF2108950C94C0
:1043B000D6210C94D7210C94D6210C94D6210C94A0
:1043C000D621CF930E94DD210E9438170E94DB2165
:1043D000C0E08C2F0E942D16811104C0CF5FCB301E
:1043E000C1F701C081E0CF91089508951F920F9207
:1043F0000FB60F9211248F939F93AF93BF93809129
:10440000EE02811113C080912F0390913003A0918F
:104410003103B09132034196A11DB11D80932F034A
:1044200090933003A0933103B0933203BF91AF91C7
:104430009F918F910F900FBE0F901F9018958091B4
:104440003703843031F10E9487071092EE0220E496
:1044500088E190E00FB6F894A895809360000FBEB5
:104460002093600083B7817F846083BF83B78160BE
:1044700083BF7894889583B78E7F83BF0FB6F894F7
:10448000A895809160008861809360001092600020
:104490000FBE08950E94130C0C948B0782E084BD1C
:1044A00093E095BD9AEF97BD80936E0008952FB766
:1044B000F89480912F0390913003A0913103B09133
:1044C00032032FBF08952FB7F89460912F03709196
:1044D000300380913103909132032FBF08959C01E6
:1044E0004FB7F89480912F0390913003A09131033E
:1044F000B09132034FBF821B930B089578941F92A3
:104500000F920FB60F9211248F939F93AF93BF9387
:1045100080912F0390913003A0913103B091320329
:104520000196A11DB11D80932F0390933003A0939A
:104530003103B0933203BF91AF919F918F910F9050
:104540000FBE0F901F901895F89481E08093E000C3
:1045500080E28093D800E9ECF0E010828FE19EE4E5
:104560000197F1F700C000001DBA109268001CBC52
:1045700010BE1FBA10927A0010926E0010926F0057
:1045800010927100109272001082ECEBF0E0108239
:1045900014B817B81AB81DB810BA108215B818B8E0
:1045A0001BB81EB811BA0C94003F089580911503F2
:1045B0000895089522E02093E9002FEF3091E8005C
:1045C000215035FD06C035ED3A95F1F70000211177
:1045D000F5CF2091E80025FF0BC040E050E066E0F9
:1045E00070E00E94D7258091E8008E778093E800E4
:1045F0000895CF93DF9320911801222339F0209161
:10460000170327FF03C060E222E002C068E021E058
:104610002093E9002FEF3091E800215035FD06C0CE
:1046200035ED3A95F1F700002111F5CF2091E80022
:1046300025FF1DC0EC0180911801811105C040E0EB
:1046400050E068E070E003C070E040E050E0CE0170
:104650000E94D7258091E8008E778093E80080E261
:10466000FE01A5EFB2E001900D928A95E1F7DF918E
:10467000CF9108958093F1027093F3026093F20258
:1046800080913703843001F582E08093E9008FEF59
:104690009091E800815095FD06C095ED9A95F1F74F
:1046A00000008111F5CF8091E80085FF0DC040E04A
:1046B00050E063E070E081EF92E00E94D7258091A6
:1046C000E8008E778093E8000895BC0184E00C94A4
:1046D0003A23BC0183E00C943A238EED99E00E94CA
:1046E000F60580913603811109C00E9468270E9457
:1046F000C5278091E20084608093E20008958AEDEE
:1047000099E00E94F60510923603089586ED99E02F
:104710000E94F6050C94D42182ED99E00E94F605E2
:104720006091330381E0611101C080E00C94BF21EE
:104730008EEC99E00E94F6059091370381E0943069
:1047400009F080E0609133030C94C4212091F002C1
:104750002F5F822F62E30E94742A992319F020931D
:10476000F00208951092F0028091F402882371F112
:1047700080913703843041F58091E9008F7020915A
:10478000EC00922F917020FD90E8892B93E090939C
:10479000E9009091EB0090FF14C09091EE0097FF1C
:1047A00010C09091E80095FF03C01092F100F9CF7E
:1047B0009091E80090FF05C09091E8009E7790935B
:1047C000E8008F708093E9001092F402089542E0AF
:1047D00061EC81E00E94E12642E261EC82E00E940D
:1047E000E12642E261EC83E00E94E12690913703EA
:1047F00081E0943009F080E0609133030C94CD2186
:1048000080913903833009F461C030F4813071F054
:10481000823009F49AC008958A3009F486C08B303A
:1048200009F46CC0893009F0A8C020C08091380319
:10483000813A09F0A2C08091E800877F8093E80068
:1048400080913C0390913D03892B21F460E285EF38
:1048500092E003C060E080E090E070E00E942226D9
:104860008091E8008B778093E80008958091380369
:10487000813209F082C080913C0390913D03029700
:1048800008F07BC08091E800877F8093E8008091EA
:10489000E80082FD05C0809137038111F8CF6DC01B
:1048A0002091F3008091F20090E0922B029731F476
:1048B0008091F100813011F0863021F48091F10077
:1048C000809315038091E8008B7753C08091380363
:1048D000813A09F052C080913C0390913D03892BAD
:1048E00009F04BC08091E800877F8093E8008091B9
:1048F000E80080FFFCCF8091180136C0809138031A
:104900008132D9F580913C0390913D03892BA9F523
:104910008091E800877F8093E8000E9416278091AD
:104920003A03809318010C94130C80913803813260
:1049300021F58091E800877F8093E8000E94162788
:1049400080913B0380931603089580913803813A48
:10495000A1F48091E800877F8093E8008091E800CF
:1049600080FFFCCF809116038093F1008091E800D6
:104970008E778093E8000C94162708959FB7F894DB
:104980001092F4029FBF90913703943009F057C002
:104990009091E9009F703091EC00232F217030FD41
:1049A00020E8922B23E02093E9002091EB0020FFE8
:1049B00043C02091EE0027FF3FC02091EF02222349
:1049C00021F02091E80025FF37C01092EF0226E089
:1049D0003091E80035FD15C030913703343061F572
:1049E0003091EB0035FD28C0215021F481E0809307
:1049F000EF0222C0EFE9FFE03197F1F700C00000BD
:104A0000E7CF8093F1008091E80085FD0AC0809196
:104A1000E80080FFFCCF8091E8008E778093E8006B
:104A200006C08FB7F89421E02093F4028FBF9F70E7
:104A30009093E90080E008959F709093E9008FEFD4
:104A4000089584B7877F84BF0FB6F894A8958091A6
:104A50006000886180936000109260000FBE90E05B
:104A600080E80FB6F89480936100909361000FBEC8
:104A70000C94CF210E9468270E94C527E2EEF0E047
:104A800080818460808378940C94592A8CE091E032
:104A90000C943C20809137038530C9F48AEC99E06E
:104AA0000E94F60580913703853079F40E941F2219
:104AB000809135038823B1F30E94E121882391F38B
:104AC0000E94C1250E94130CEDCF0C944A22089538
:104AD00008950C946B25292F332723303105C9F015
:104AE00060F42130310581F02230310509F041C0F8
:104AF0008BE590E020E13AE040C021323105E1F061
:104B00002232310531F135C082E190E02BE63AE006
:104B100034C099278130910549F028F0029749F572
:104B2000E2EEF9E005C0ECE0FAE002C0ECEFF9E0FB
:104B3000849190E09F0121C063307105D0F4660F2D
:104B4000771FFB01EC50FE4F2081318189E090E01E
:104B500014C06330710568F4FB01EE0FFF1FE251D2
:104B6000FE4F20813181FB01E551FE4F808190E0B5
:104B700004C080E090E020E030E0FA01318320833F
:104B8000089580E189BD82E189BD09B400FEFDCFB1
:104B90008091D8008F7D8093D8008091E000826062
:104BA0008093E0008091E00081FDFCCF0895CF92DA
:104BB000DF92EF92FF920F931F93CF93DF93EC015D
:104BC0008B017A010E943527811133C0E114F10471
:104BD00039F0F70180819181081B190BC80FD91F8B
:104BE000C12CD12C0115110519F18091E80085FD2A
:104BF00016C08091E8008E778093E800E114F104FC
:104C000049F0F70180819181C80ED91ED182C082FE
:104C100085E00FC00E943527882321F30AC08991BF
:104C20008093F10001501109FFEFCF1ADF0ADACFAC
:104C300080E0DF91CF911F910F91FF90EF90DF9077
:104C4000CF90089520913E0330913F0326173707F8
:104C500048F06115710539F42091E8002E77209312
:104C6000E80001C0B901FC0120E06115710579F18E
:104C7000809137038823F1F18530F1F18091E800CC
:104C800083FD3CC08091E80082FD2EC08091E80049
:104C900080FFEBCF2091F3008091F20090E0922B07
:104CA0006115710551F08830910538F421912093F8
:104CB000F100615071090196F3CF21E0089709F0E6
:104CC00020E08091E8008E778093E800CECF21111C
:104CD000CFCF0AC080913703882361F0853061F01F
:104CE0008091E80083FD0AC08091E80082FFF2CF46
:104CF00080E0089582E0089583E0089581E00895BA
:104D000020913E0330913F032617370748F0611585
:104D1000710539F42091E8002E772093E80001C056
:104D2000B901FC0120E06115710591F18091370313
:104D3000882309F440C0853009F43FC08091E80021
:104D400083FD3DC08091E80082FD2FC08091E80086
:104D500080FFE9CF2091F3008091F20090E0922B48
:104D60006115710559F08830910540F42491209324
:104D7000F1003196615071090196F2CF21E0089758
:104D800009F020E08091E8008E778093E800CBCF97
:104D90002111CCCF0AC080913703882361F0853080
:104DA00061F08091E80083FD0AC08091E80082FFF5
:104DB000F2CF80E0089582E0089583E0089581E0D5
:104DC0000895982F973068F59093E900981739F077
:104DD0007091EC002091ED005091F00003C0242F61
:104DE000762F50E021FD02C09F5FECCF3091EB00A9
:104DF0003E7F3093EB003091ED003D7F3093ED002E
:104E00003091EB0031603093EB007093EC00209315
:104E1000ED005093F0002091EE0027FDE5CF80E0FB
:104E200008958F708093E90081E0089580913803A0
:104E300087FF11C08091E80082FD05C08091370393
:104E40008111F8CF11C08091E8008B770BC0809161
:104E50003703882349F08091E80080FFF8CF8091E4
:104E6000E8008E778093E80008952091E400309167
:104E7000E50095E64091EC00842F817040FF23C04F
:104E80008091E80080FD1DC080913703882399F050
:104E9000853099F08091EB0085FD11C04091E400D0
:104EA0005091E5002417350729F3915011F09A012C
:104EB000E1CF84E0089582E0089583E0089581E0E1
:104EC000089580E008954091E80042FFDDCF089505
:104ED0000E94D6270E94DE27E0EEF0E0808181600C
:104EE0008083E8EDF0E080818F77808319BCA7EDA7
:104EF000B0E08C918E7F8C9380818F7E8083109226
:104F0000360308950F931F93CF93DF930E94D62704
:104F10000E94DE27C8EDD0E088818F778883888162
:104F20008068888388818F7D888319BC10923703BD
:104F300010923303109235031092340300EE10E008
:104F4000F80180818B7F808388818160888342E043
:104F500060E080E00E94E126E1EEF0E080818E7F5B
:104F60008083E2EEF0E080818160808380818860D0
:104F70008083F80180818E7F80838881806188832F
:104F8000DF91CF911F910F910895E8EDF0E08081BE
:104F90008F7E8083E7EDF0E080818160808384E014
:104FA00082BF81E0809336030C948227E8EDF0E025
:104FB00080818E7F80831092E20008951092DA0043
:104FC0001092E10008951F920F920FB60F921124D4
:104FD0002F933F934F935F936F937F938F939F9301
:104FE000AF93BF93EF93FF938091E10082FF0BC0DB
:104FF0008091E20082FF07C08091E1008B7F809367
:10500000E1000E94A6238091DA0080FF1FC08091FA
:10501000D80080FF1BC08091DA008E7F8093DA0079
:105020008091D90080FF0DC080E189BD82E189BDFA
:1050300009B400FEFDCF81E0809337030E946D2309
:1050400005C019BC109237030E947F238091E100B4
:1050500080FF19C08091E20080FF15C08091E200BE
:105060008E7F8093E2008091E20080618093E20075
:105070008091D80080628093D80019BC85E080932D
:1050800037030E948C238091E10084FF30C080911F
:10509000E20084FF2CC080E189BD82E189BD09B4B2
:1050A00000FEFDCF8091D8008F7D8093D800809145
:1050B000E1008F7E8093E1008091E2008F7E8093FB
:1050C000E2008091E20081608093E20080913303EE
:1050D000882311F084E007C08091E30087FD02C0BF
:1050E00081E001C083E0809337030E949823809180
:1050F000E10083FF29C08091E20083FF25C08091F9
:10510000E100877F8093E10082E080933703109273
:1051100033038091E1008E7F8093E1008091E20073
:105120008E7F8093E2008091E20080618093E200B4
:1051300042E060E080E00E94E1268091F00088601B
:105140008093F0000E948623FF91EF91BF91AF9171
:105150009F918F917F916F915F914F913F912F918F
:105160000F900FBE0F901F9018951F920F920FB6C1
:105170000F9211242F933F934F935F936F937F93DD
:105180008F939F93AF93BF93CF93DF93EF93FF934F
:10519000C091E900CF708091EC00D82FD17080FDD4
:1051A000D0E81092E9008091F000877F8093F000B2
:1051B00078940E94F9281092E9008091F0008860AC
:1051C0008093F000CD2BCF70C093E900FF91EF9159
:1051D000DF91CF91BF91AF919F918F917F916F910F
:1051E0005F914F913F912F910F900FBE0F901F90A5
:1051F00018951F93CF93DF93CDB7DEB7AA970FB65D
:10520000F894DEBF0FBECDBFE8E3F3E08091F1007C
:10521000819323E0E034F207C9F70E9400248091D3
:10522000E80083FF2EC18091380390913903492F04
:1052300050E04A30510508F024C1FA01EF55FF4F04
:105240000C94942A803821F0823809F01AC108C0E1
:105250008091340390913503992389F082600FC0C7
:1052600080913C038F70873008F00BC18093E90078
:105270008091EB0085FB882780F91092E9009091DE
:10528000E800977F9093E8008093F1001092F1007E
:10529000D1C0282F2D7F09F0F4C0882319F0823067
:1052A00061F0EFC080913A03813009F0EAC0933099
:1052B00009F080E0809335032EC080913A0381117C
:1052C0002AC080913C038F702FEF280F263008F002
:1052D000D8C08093E9002091EB0020FF1CC09330E0
:1052E00021F48091EB00806214C09091EB009061FA
:1052F0009093EB0021E030E0A90102C0440F551F5C
:105300008A95E2F74093EA001092EA008091EB0060
:1053100088608093EB001092E9008091E800877F1D
:105320008093E8000E941627ACC08111AAC010919A
:105330003A031F778091E3008078812B8093E3000C
:105340008091E800877F8093E8000E941627809173
:10535000E80080FFFCCF8091E30080688093E30049
:10536000111102C082E001C083E08093370389C03D
:105370008058823008F085C080913A0390913B03B9
:105380008C3D53E0950779F583E08A838AE289832F
:105390004FB7F894DE01139620E03EE051E2E32F90
:1053A000F0E050935700E49120FF03C0E295EF70C6
:1053B0003F5FEF708E2F90E0EA3010F0C79601C08B
:1053C000C0968D939D932F5F243149F74FBF8091F5
:1053D000E800877F8093E8006AE270E0CE010196E2
:1053E0000E94222616C060913C0370913D03AE01DD
:1053F0004F5F5F4F0E946925BC01892B09F441C0B2
:105400009091E800977F9093E80089819A810E94AB
:1054100080268091E8008B778093E80032C0803846
:1054200081F58091E800877F8093E80080913303C5
:105430008093F1008091E8008E7772CF811121C0B6
:1054400080913A0390913B0399270297D4F480917D
:10545000E800877F8093E80080913A0380933303CC
:105460000E94162780913303811106C08091E300CA
:1054700087FD02C081E001C084E0809337030E9471
:10548000E7238091E80083FF0AC08091E800877FCE
:105490008093E8008091EB0080628093EB00AA96F5
:1054A0000FB6F894DEBF0FBECDBFDF91CF911F9135
:1054B0000895CF93809137038823A1F0C091E9002C
:1054C000CF709091EC00892F817090FD80E8C82BFF
:1054D0001092E9008091E80083FD0E94F928CF70C6
:1054E000C093E900CF910895991B79E004C0991FFA
:1054F000961708F0961B881F7A95C9F7809508952E
:1055000097FB072E16F4009407D077FD09D00E9470
:105510009A2A07FC05D03EF4909581959F4F0895F7
:10552000709561957F4F0895EE0FFF1F0590F491E0
:10553000E02D0994AA1BBB1B51E107C0AA1FBB1F8A
:10554000A617B70710F0A61BB70B881F991F5A950F
:10555000A9F780959095BC01CD010895FB01DC0170
:1055600004C08D910190801921F441505040C8F73A
:10557000881B990B0895F999FECF92BD81BDF89AC9
:10558000992780B50895A8E1B0E042E050E00C947E
:10559000EF2A262FF999FECF92BD81BDF89A019787
:1055A00000B4021639F01FBA20BD0FB6F894FA9A6B
:1055B000F99A0FBE08950396272F0E94CA2A0E94C7
:1055C000C92A252F0E94CA2A242F0C94CA2A019680
:1055D000272F0E94CA2A0C94C92ADC01CB01FC01A6
:1055E000F999FECF06C0F2BDE1BDF89A319600B43C
:0E55F0000D9241505040B8F70895F894FFCF47
:1055FE00C8009702280850011E0A1401D622F9226B
:10560E00DA2269236523D92201E200E900EA00B516
:10561E0000B600B700CD008301CC008A0192019440
:10562E00012102230224022502260227022A02B3A6
:10563E0000B4006F007000818283E200E900EA008E
:10564E00B500B600B700CD008301CC008A019201EF
:10565E0094012102230224022502260227022A0295
:10566E00B300B4006F007000818283303132339208
:10567E009367959497343536F7F6F5F4F1F03F3F8E
:10568E003F006D6B5F64656C6179006D6B5F696E79
:10569E0074657276616C006D6B5F6D61785F7370AF
:1056AE00656564006D6B5F74696D655F746F5F6DCA
:1056BE006178006D6B5F776865656C5F6D61785FB3
:1056CE007370656564006D6B5F776865656C5F749C
:1056DE00696D655F746F5F6D61780040B622550B22
:0A56EE009F0A7D0A220A3B0A540AB3
:00000001FF
